:10000000A8C00000C1C00000BFC00000BDC000000B
:10001000BBC00000B9C00000B7C00000B5C0000000
:10002000B3C00000B1C00000AFC00000F3C30000C7
:10003000ABC00000A9C00000A7C00000A5C0000020
:10004000A3C00000A1C000009FC000009DC0000030
:100050009BC0000099C0000097C0000062C1000072
:1000600093C0000091C000008FC000008DC0000050
:100070008BC0000089C0000087C0000085C0000060
:1000800083C0000081C000007FC000007DC0000070
:100090007BC0000079C0000005010906A1017501BF
:1000A0009508050719E029E715002501810295014A
:1000B0007508810395057501050819012905910247
:1000C00095017503910395067508150025650507CB
:1000D000190029658100C01201100100000008EB21
:1000E0000342200000010200010902220001010078
:1000F000C0320904000001030101000921110100BF
:1001000001223F000705810308000A0403090416C1
:10011000034C00650020004100760065006E00671A
:100120000065007200000028034300720061007A3D
:10013000007900200054006F006E00790020004B11
:10014000006500790062006F0061007200640000C9
:10015000000011241FBECFEFD2E0DEBFCDBF11E003
:10016000A0E0B1E0E8ECFFE002C005900D92AE30F7
:10017000B107D9F711E0AEE0B1E001C01D92AE3A8F
:10018000B107E1F74ED01EC73BCFBF92CF92DF92AF
:10019000EF92FF920F931F93CF93DF9384B7877FE4
:1001A00084BF28E10FB6F89420936000109260009D
:1001B0000FBE3CECC32ED12C87E690E0F601918374
:1001C00080839AECE92EF12C86E0B82EF701B082FC
:1001D00008EC10E0F8011082C9ECD0E02883539AB3
:1001E0005A9A0DD384E085BD5F9A579A1882F80118
:1001F0001082F70110828FEC90E0F60191838083EA
:10020000F701B08282E0F801808388E98883DF917A
:10021000CF911F910F91FF90EF90DF90CF90BF9003
:1002200008950F931F93B1DF2FB7F8948FE191E0FA
:100230009093A00180939F019093A2018093A101CC
:100240002FBF78948C019FB7F8948091A3019FBF32
:10025000883048F1A89AAEE0B1E0E091A101F091B8
:10026000A2019191F093A201E093A10181E0EF3905
:10027000F80721F40093A1011093A2012FB7F8947D
:100280008091A30181508093A3012FBF9D9381E0B2
:10029000A631B80711F7809116019091C80095FF1B
:1002A000FCCF8093CE0080E091E0B6D553D4CBCF85
:1002B0000895089580E091E087D5E2EEF0E0808136
:1002C00084608083089580E091E056C480910B01A2
:1002D00090910C01009729F0019790930C01809365
:1002E0000B0108950F931F93CF93DF93E801EEE086
:1002F000F1E0822F932FDC0181918D9381E0E63133
:10030000F807D1F788E090E09983888380E0DF9157
:10031000CF911F910F910895F9018081809316016B
:1003200008951F920F920FB60F9211242F938F935F
:100330009F93EF93FF938091CE009EB39430F9F496
:10034000E0919F01F091A0018083E0919F01F091E5
:10035000A001CF0101969093A00180939F0121E01D
:100360008F39920721F48FE191E0928381839FB7C7
:10037000F8948091A3018F5F8093A3019FBFFF91A9
:10038000EF919F918F912F910F900FBE0F901F9023
:100390001895933089F0943028F4913059F19230C7
:1003A00071F505C09132E1F0923249F51EC022E2AA
:1003B00030E0E9EEF0E027C0813049F0813018F0FC
:1003C0008230E9F408C0EBE0F1E0249107C0EFE0EF
:1003D000F1E0249103C0E7E2F1E0249130E013C0A2
:1003E00029E030E0EBEFF0E00EC02FE330E0E8E989
:1003F000F0E009C022E130E0E7EDF0E004C020E0E9
:1004000030E0E0E0F0E0DA011196FC93EE93C901F0
:10041000089528E030E040E003C04F5F220F331F13
:1004200028173907D0F3842F8295807F0895809311
:10043000E900EBEEF0E0808181608083EDEEF0E09A
:1004400010826093EC0040838091EE00881F882723
:10045000881F08951092F40080E08093E9001092C4
:10046000F0001092E8001092ED009091EB009E7F5A
:100470009093EB008F5F853081F708958091A601FE
:1004800087FF11C003C08EB38823B1F08091E800CC
:1004900082FFF9CF8091E8008B778093E800089580
:1004A0008EB3882349F08091E80080FFF9CF8091D6
:1004B000E8008E778093E800089584E69091EC0040
:1004C00090FF05C09091E80090FF05C01BC090917F
:1004D000E80092FD17C09EB39923B1F09EB395300A
:1004E000A9F09091EB0095FD13C09091E10092FF6F
:1004F000E5CF9091E1009B7F9093E100882351F03C
:100500008150DCCF80E0089582E0089583E0089573
:1005100081E0089584E00895AF92BF92DF92EF9258
:10052000FF920F931F93DF93CF930F92CDB7DEB758
:10053000082F5B017A019983C0DFD82E9981882327
:1005400031F5192F1CC08091E80085FD10C0809105
:10055000E8008E778093E800E114F10421F0F701C0
:100560000995813081F0A9DF882349F00FC0F80197
:1005700081918F018093F1000894A108B108A11422
:10058000B10409F704C075E0D72E01C0D82E8D2D17
:100590000F90CF91DF911F910F91FF90EF90DF901F
:1005A000BF90AF900895282F392FF9018091AC01A9
:1005B0009091AD018617970718F4BC0190E032C006
:1005C00061157105D9F78091E8008E778093E80076
:1005D000F5CF8091E80083FD37C08091E80082FD6F
:1005E0002DC08EB38823A1F18EB3853079F180912F
:1005F000E80080FF17C08091F20006C091919093AF
:10060000F100615070408F5F6115710511F0883005
:10061000A8F391E0883009F090E08091E8008E77AF
:100620008093E80061157105A1F6992391F606C043
:100630008EB3882369F08EB3853061F08091E80035
:1006400082FFF6CF80E0089581E0089583E0089569
:1006500082E0089583E00895282F392FC901209161
:10066000AC013091AD012617370718F4B90130E01D
:1006700034C061157105D9F72091E8002E772093D9
:10068000E800F5CF2091E80023FD39C02091E80073
:1006900022FD2FC02EB32223B1F12EB3253089F1D4
:1006A0002091E80020FF19C02091F20008C0FC0151
:1006B0000196E491E093F100615070402F5F611565
:1006C000710511F0283098F331E0283009F030E05E
:1006D0002091E8002E772093E8006115710591F6CE
:1006E000332381F606C08EB3882369F08EB385303C
:1006F00061F08091E80082FFF6CF80E0089581E00C
:10070000089583E0089582E0089583E008956115D7
:10071000710519F51DC02091E80023FD2EC02EB3F0
:10072000222379F12EB3253051F12091E80022FFE8
:10073000F2CFE82FF92F07C08091F1008193CF010C
:100740006150704029F0CF012091F2002223A1F7DF
:100750002091E8002B772093E80061157105D9F608
:1007600006C08EB3882369F08EB3853061F0809126
:10077000E80080FFF6CF80E0089581E0089583E0EF
:10078000089582E0089583E008953ED040D01EBAD7
:100790001092A40184E089BD89B5826089BD09B445
:1007A00000FEFDCF8091D800982F9F779093D800BE
:1007B00080688093D800809163008E7F809363006F
:1007C0008091D8008F7D8093D8008091E0008E7F4B
:1007D0008093E0008091E1008E7F8093E100809122
:1007E000E20081608093E2008091E100877F809346
:1007F000E1008091E20088608093E2000895C5DF07
:1008000081E08093A50108951092E200089510926E
:10081000E10008951F920F920FB60F9211242F93AB
:100820003F934F935F936F937F938F939F93AF9378
:10083000BF93EF93FF938091E10080FF1BC08091F5
:10084000E20080FF17C08091E1008E7F8093E1007D
:100850008091E2008E7F8093E2008091E2008061CF
:100860008093E2008091D80080628093D80019BC08
:100870001EBA1FDD8091E10084FF29C08091E20053
:1008800084FF25C084E089BD89B5826089BD09B433
:1008900000FEFDCF8091D8008F7D8093D80080919D
:1008A000E1008F7E8093E1008091E2008F7E809353
:1008B000E2008091E20081608093E2008091A401D7
:1008C000882311F084E001C081E08EBBF1DC8091CF
:1008D000E10083FF22C08091E20083FF1EC080916F
:1008E000E100877F8093E10082E08EBB1092A4013B
:1008F0008091E1008E7F8093E1008091E2008E7F05
:100900008093E2008091E20080618093E200A2DDAA
:1009100080E060E042E08BDD1CD18091E10082FF4D
:100920000AC08091E20082FF06C08091E1008B7FC7
:100930008093E100CBDCFF91EF91BF91AF919F914C
:100940008F917F916F915F914F913F912F910F9078
:100950000FBE0F901F9018951F93DF93CF9300D079
:10096000CDB7DEB7E6EAF1E08091F100819381E056
:10097000EE3AF807C9F78091A6019091A70195304A
:1009800009F46BC0963040F4913061F1913070F011
:10099000933009F0C9C026C0983009F49BC0993043
:1009A00009F4AAC0963009F0BFC075C0803809F4B8
:1009B000BCC0823809F0B8C08091AA0187708093CA
:1009C000E9009091EB001092E9008091E800877FA8
:1009D0008093E80081E095FF80E08093F100109221
:1009E000F10083C0882319F0823009F09DC08F7117
:1009F000823009F09AC08091A801882341F52091A6
:100A0000AA01277009F491C02093E9008091EB00BE
:100A100080FF8BC08091A701833021F48091EB008F
:100A2000806213C08091EB0080618093EB0081E0D5
:100A300090E002C0880F991F2A95E2F78093EA00A0
:100A40001092EA008091EB0088608093EB00109296
:100A5000E9008091E800877F4BC0882309F064C0DB
:100A60001091A8018091E800877F8093E80006DD5F
:100A700004C08EB3882309F458C08091E80080FF39
:100A8000F8CF1F7711F083E001C082E08EBB1068C1
:100A90001093E3004AC08058823008F045C080912E
:100AA000A8019091A9016091AA01AE014F5F5F4F2B
:100AB00070DCBC010097C9F18091E800877F8093CA
:100AC000E80089819A81C8DD8091E8008B77809366
:100AD000E8002BC0803841F58091E800877F809343
:100AE000E8008091A4018093F1008091E8008E7766
:100AF0008093E800C3DC19C08823B1F49091A80169
:100B0000923098F48091E800877F8093E80090937A
:100B1000A401B4DC8091A401882311F084E001C019
:100B200083E08EBBC7DB01C0CEDB8091E80083FF92
:100B30000AC08091EB0080628093EB008091E80016
:100B4000877F8093E8000F900F90CF91DF911F91E6
:100B5000089508951F938EB3882361F01091E900E2
:100B600017701092E9008091E80083FF01C0F4DE65
:100B70001093E9001F9108956F927F928F929F9238
:100B8000AF92BF92CF92DF92EF92FF920F931F939B
:100B9000DF93CF9300D00F92CDB7DEB77C016DB657
:100BA0007EB68091E80083FFF8C0F701808190E075
:100BB0002091AA013091AB012817390709F0EDC047
:100BC0008091A701833009F499C0843030F48130DA
:100BD00071F0823009F0E1C0C8C08A3009F4AEC0BB
:100BE0008B3009F498C0893009F0D7C04CC080918F
:100BF000A601813A09F0D1C0CDB6DEB69DB68D2CE6
:100C00008091E800877F8093E8001B821A828091A0
:100C1000A8010091A9018983F7014781C41AD1086D
:100C20000FB6F894DEBE0FBECDBE0894C11CD11C19
:100C3000BC2CAD2CC60160E070E050E0BCD1402F70
:100C40004150C701BE016F5F7F4F96018E010E5F5D
:100C50001F4F48DBF701258136812115310529F029
:100C60004781C901B60150E09DD11092E9006A8127
:100C70007B818B2D9A2D97DC8091E8008B77809378
:100C8000E800940133C08091A601813209F085C04B
:100C9000CDB6DEB6BDB6AD2C8091E800877F8093DF
:100CA000E8000091AC011091AD019090A8018090F6
:100CB000A9018DB79EB7801B910B0FB6F8949EBF0C
:100CC0000FBE8DBFCDB6DEB60894C11CD11CC601C7
:100CD000B8011DDD482D4150C701692D96011CDB6F
:100CE0008091E8008E778093E8009501832F922F02
:100CF0000FB6F8949EBF0FBE8DBF4FC08091A60166
:100D0000813A09F04AC08091E800877F8093E8002B
:100D1000F70180853AC08091A601813209F03DC07B
:100D20008091E800877F8093E8009091A80181E09E
:100D3000992309F480E0F70180872EC08091A601F5
:100D4000813259F58091E800877F8093E800809197
:100D5000A8019091A901807036E0969587953A9503
:100D6000E1F7F7019287818717C08091A601813A48
:100D7000A1F48091E800877F8093E800F7018185E6
:100D8000928596958795969587958093F1008091A9
:100D9000E8008E778093E80071DB0FB6F8947EBE92
:100DA0000FBE6DBE0F900F900F90CF91DF911F91EE
:100DB0000F91FF90EF90DF90CF90BF90AF909F90FA
:100DC0008F907F906F9008950F931F93CF93DF9331
:100DD000FC010896DC0185E0ED0119928A95E9F79E
:100DE00081E0808784EF91E092878187228133813F
:100DF00001818481882311F014E001C010E0C90151
:100E000008DB412F482B4260802F61EC10DBDF9123
:100E1000CF911F910F9108954F925F926F927F92A1
:100E20008F929F92AF92BF92CF92DF92EF92FF92FA
:100E30000F931F93DF93CF9300D00F92CDB7DEB700
:100E40007C016DB67EB68EB3843009F085C0F701A3
:100E500081818093E9008091E80085FF7DC05DB6C7
:100E6000472C4781CDB6DEB6C41AD1080FB6F89428
:100E7000DEBE0FBECDBE0DB71EB70F5F1F4FB02E2B
:100E8000912E19821B821A82C80160E070E050E046
:100E900092D0C701BE016F5F7F4F40E098018E0185
:100EA0000E5F1F4F1FDA882EF7018185928500970C
:100EB00059F081E090E0238534852115310511F04A
:100EC00080E090E06C0102C0CC24DD24F7010581B4
:100ED00016810115110599F04A815B818B2D992DA1
:100EE000B80153D0AA24A394009709F4AA24F701C7
:100EF0004781C8016B2D792D50E054D001C0AA2440
:100F00008A819B81009701F1882029F4AA2019F495
:100F1000C114D104C9F0F701818592859487838734
:100F200081818093E9008981882311F08093F10009
:100F30006A817B818B2D992D40E050E0EDDA809124
:100F4000E8008E778093E8009201832F942D0FB6EE
:100F5000F8949EBF0FBE8DBF0FB6F8947EBE0FBE35
:100F60006DBE0F900F900F90CF91DF911F910F9159
:100F7000FF90EF90DF90CF90BF90AF909F908F90B9
:100F80007F906F905F904F900895FB01DC0104C04B
:100F90008D910190801921F441505040C8F7881B71
:100FA000990B0895FB01DC0102C001900D924150A4
:100FB0005040D8F70895DC0101C06D934150504076
:080FC000E0F70895F894FFCF5B
:0E0FC8000001080000170108000000000000F2
:00000001FF
